S018000064656D6F70726F675F786D63313430302E7372656343
S3151000300000400020A1400010000000000000000059
S315100030100018040000010000EE11AA5500B5E221C7
S3151000302049004058C02189000140002901D10120E2
S3151000303000E00020C0B200BD30B4C9B2D2B2140450
S315100030400C43DBB21D062543E2246400055130BC57
S315100030507047016840220A430260704701684022A7
S3151000306091430160704700B5814200D3080000BD4E
S3151000307000B5884200D3080000BDF1B588B00E0037
S315100030800C250C24002007900120059000200690A6
S31510003090002004909B48009001200500412D4BD242
S315100030A030680A214843290000F006FA0390039875
S315100030B0716800F001FA070038000A2100F007FADB
S315100030C0062906D338000A2100F0F6F907007F1CFE
S315100030D004E038000A2100F0EFF90700002F06D0AF
S315100030E003980A21794300F0E7F9029006E0039865
S315100030F00A2100F0E1F90290012007000298716898
S31510003100884204D302987168401A019003E07068EF
S315100031100299401A0190152F0CD2019800998842F5
S3151000312008D207950497019800900198FA21890012
S31510003130884201D36D1CB1E772480090402004000C
S31510003140032C1AD32000401C6E494843049900F002
S31510003150B3F93289904203D33289821A110002E000
S315100031603289121A1100009A914201D205940091E7
S315100031703289904201D3641EE2E704980599401AF9
S31510003180401E06900898FFF764FF0698401E01033C
S31510003190E020C00108407189491E8A01C0211140F2
S315100031A001430598401E0002F022120102400A4314
S315100031B00798401E8006800E1043089908610898EB
S315100031C0FFF74CFF09B0F0BD70B505000C001600F6
S315100031D02800FFF723FF0028FAD023005B1CDBB280
S315100031E03200D2B202212800FFF726FF70BD10B5BB
S315100031F004008020800300F098F92068012188439C
S31510003200206020688007FCD410BD38B5040020006B
S3151000321000F085F8012802D0022804D007E000F05B
S3151000322097F9050005E000F09DF9050001E0002082
S315100032300500280032BDF6B589B006003000FFF74C
S31510003240D6FF09A80178300000F05EF83000FFF7CD
S31510003250DCFF01908021C900009101980A9900F0C5
S315100032602BF90099091A0020FFF7FDFE6F49FFF7A9
S31510003270FFFE059001988021C900059A891A00F071
S315100032801BF907900A988009069001988009029008
S315100032906649009106988021C9004843029900F0BA
S315100032A00BF90099FFF7E4FE04900298049948433D
S315100032B0800A0700BF010A98C01B0A99079A891A43
S315100032C0884201D3012400E00024E4B2002C02D08D
S315100032D00598039001E004980390E4B2002C01D005
S315100032E0012500E00225F06851490140F160F068BF
S315100032F0EDB2A903039A0A430243F2600BB0F0BD84
S315100033000000000010270000E422520082580F230C
S315100033109A43C9B20A43E4235B00C2507047E421C2
S31510003320490040580007000F7047F8B504002068A0
S315100033305C4940184709780940033902F826760196
S315100033400E40064320688068574901402068816016
S31510003350206880683043216888606068800002D5E4
S31510003360606880003BD5207E002802D0207E012890
S3151000337035D120202168C861606801008900C90F15
S31510003380002914D1606805006D0F6D07290060686B
S3151000339085040D4320688561A06805006D0F6D07D3
S315100033A02900A06885040D432068C56005E06068A3
S315100033B021688861A0682168C860207E012807D12D
S315100033C0200000F00DF8802000052168C86103E098
S315100033D0802000012168C86134482168C861F1BDA8
S315100033E010B5010003200A7E012A1AD120220B688B
S315100033F0DA610A6812682E4B13400A7B1206F02413
S31510003400240514401C430A6814600A690B681A6183
S315100034104A690B685A61274A0B68DA610022100064
S3151000342001E003221000C0B210BD0000FF0300002F
S31510003430003CFFFFF0B501000120002200230C68BC
S31510003440E5692C002405E40F0D68EE6935006D075B
S31510003450ED0F002C02D00326300020E0012D02D102
S31510003460022630001BE00E6836690E610E6876691A
S315100034704E610E68F669B6083700FF07FF0F3A006F
S315100034800E68F669F6083700FF07FF0F3B00D2B249
S31510003490002A02D0DBB2002BE5D100263000C0B2E4
S315100034A0F0BD000000F0FBAFFF00FFFF4000A006DC
S315100034B0FFFFFFF040002800020004200F4B1860A9
S315100034C00F4802600F48016010480068704770B5D9
S315100034D002000B00042009490860094802600948E7
S315100034E003600948006800210100002004000D0057
S315100034F00648006800212043294370BD340003406C
S3151000350020000340240003402C0003402800034001
S31510003510C3200E490860704700B5C0200B490860EB
S315100035200A4800684007FBD400BD10B50400FFF739
S31510003530F3FF0A48006820430849086006480068F7
S315100035404000FBD4FFF7E4FF10BD0000240001404B
S315100035500348006870470000000301401003014053
S31510003560D401002000487047002D310100B5BFF38B
S315100035704F8F8948D3490860BFF34F8F00BFFDE7CF
S3151000358010B4C9B204234B43C318DB690724A34301
S31510003590D2B21343C9B204244C430419E36110BCDC
S315100035A070478A2149004058C1080800C007C00F5B
S315100035B07047016C0F22914302220A43026470473E
S315100035C070B504000D001600EDB2042068432018F3
S315100035D0C06950218843EDB2042169436118C8615E
S315100035E03200D2B22900C9B22000FFF7C9FF70BD60
S315100035F0C26807239A43C9B24B075B0F1343C360D4
S315100036007047016840220A430260704701684022F1
S31510003610914301607047016801220A4302607047B6
S31510003620016801229143016070470068C0697047C4
S315100036300268D16170478168802292050A438260D0
S315100036400168C968802292050A430168CA607047FA
S3151000365080B500F00DF800F0A1F801BD80B500F0BE
S3151000366045F800F031F901BD80B5FFF77FFF01BDC8
S3151000367000B587B0E1200002009008206946087165
S3151000368008206946487101206946887110206946EC
S31510003690C8710020694608816946A54800F068F996
S315100036A000206946087505AA0321A24800F0F4F91E
S315100036B09C206946087303AA02219E4800F0ECF983
S315100036C0002200219A48FFF77BFF012304221021D4
S315100036D0974800F0BAFA012304220021944800F01A
S315100036E0CDFA9348FFF765FF07B000BD80B5924845
S315100036F00078002813D1914800F03EF801283AD1FD
S315100037008E480078002836D000F065FB8C4908609A
S3151000371001208949087000208A4908702BE08748E3
S31510003720884909784018401C00F026F8012818D15D
S3151000373084480078401C83490870824800787F4985
S315100037400978884217D100207B4908707B48407859
S31510003750FF2810D17948807800280CD1FFF784FF14
S3151000376009E000F038FB764909686431814202D2DB
S3151000377000207149087001BD10B504006C48FFF7B0
S3151000378010FF002805D16A4800F034F92070012096
S3151000379000E0002010BD00000400FA0570B588B0E6
S315100037A0FFF7D6FE04006848844202D20220444342
S315100037B0F9E76648844201D36408FAE7220001213A
S315100037C06348FFF738FD009462480190FA204001E3
S315100037D06946088101206946488169465E48FFF7B7
S315100037E04CFC5D48FFF70DFF5B48FFF714FF5B4885
S315100037F05B4908605A4840688000800880210906A5
S3151000380001435748416057480600760076085448E9
S315100038104068400F4007F100C90801435048416015
S315100038204F488068400F4007F100C90801434C48D3
S3151000383081604B4840684C490140494841604848BE
S31510003840FFF7F9FE082046490873002005002800F6
S315100038504349097BC0B2884206D200204049EDB2E6
S31510003860491908746D1CF2E700203D4908763C485A
S31510003870FFF75BFD012201213548FFF7A5FC36480D
S31510003880FFF7C4FE3448FFF7CBFE002069460875E3
S3151000389005AA0821354800F0FFF8A42069460873E8
S315100038A003AA0921314800F0F7F82B48FFF7A9FEC3
S315100038B002212948FFF79CFE2748FFF7A7FE08B00C
S315100038C070BD00000CED00E030B583B00025244833
S315100038D0FFF7ABFEC0071BD52148FFF7ABFD00284D
S315100038E012D10020040020001D49097BC0B2884275
S315100038F00AD21B48E4B20019007C6946E4B20855A6
S3151000390001200500641CEEE701211548FFF790FE23
S31510003910EDB2012D0BD10020050068460078FF2876
S3151000392005D168464078002801D1FFF79DFE37BDC6
S315100039300002004800010440D1010020540100207B
S3151000394098010020D0010020001BB700010E2707A8
S315100039500000045020A1070000030450201004505A
S31510003960A001002067060000FFFFFFDF00040440EF
S3151000397070B504000E001025200000F0EFF8F07965
S31510003980002801D0F07905002A003168200000F0E7
S3151000399005F9B079401E40002900891CC901FF2293
S315100039A09143014312480843E0633079401E0006F4
S315100039B081214900014361637079002806D0606B4C
S315100039C07179491E09040143616305E0606B317921
S315100039D0491E090401436163A020C000A0630020B2
S315100039E0C043E0640820305E206470BD0000000013
S315100039F00100030000B50100862252008A58E02318
S31510003A00DB041340002B02D14A6D100003E08E2216
S31510003A1052008A58100080B200BDF8B401684218EE
S31510003A2043685908511800918168DB0701D54B4648
S31510003A30C918009B9A4202D10C30F2BC7047137819
S31510003A40521C032403261E4002D11678F61C521C63
S31510003A501D090F2D07D115780F35521C03E0177865
S31510003A60521C0F70491C761EF9D1002DE1D0167824
S31510003A70521C9B081C40032C01D11478521C2302A3
S31510003A80F3185C420B19AD1CD3D01C785B1C0C7060
S31510003A90491C6D1ECDD0F8E7F0B5C9B28B100424C1
S31510003AA06343C318C9B28C1004256C4304192469E6
S31510003AB0FC258E07B60F08277E43B540AC431C6124
S31510003AC0436F03244D00AC40A3434367C9B2CB08F0
S31510003AD004246343C318C9B2CC0804256C430419E3
S31510003AE0246C04254E07760F04277E43B540AC435D
S31510003AF01C64C9B2CB0804246343C318C9B2CC08EA
S31510003B0004256C430419246C55784F077F0F04263F
S31510003B107743BD4025431D640F4B984204D1036E75
S31510003B2001248C40A343036653688B404360C9B29B
S31510003B308B1004246343C318C9B28C1004256C433C
S31510003B400419246915788F07BF0F08267743BD40DF
S31510003B5025431D61F0BD00000002044010B50400AD
S31510003B609020C005844202D05B48844203D15B4852
S31510003B7000F0A0F808E05A48844202D0594884421E
S31510003B8002D1594800F096F80320E060E068C007BB
S31510003B90FCD5206C0F218843206410BDF0B589B088
S31510003BA007000D001600642D48D3002E46D0FFF7EF
S31510003BB0CFFC6421FFF780FC079028006421FFF7F3
S31510003BC07BFC0500012005900120029047480090DB
S31510003BD046480400002C1DD0079860432900714305
S31510003BE0FFF76AFC04900498800A039004988005F5
S31510003BF0800D019003988021C900884208D201984F
S31510003C000099884204D20198009003980290059476
S31510003C10641EDFE70598802109020143396178693E
S31510003C2033490140701E800208430299491E090457
S31510003C300143796100206946087602E00120694651
S31510003C4008766846007E09B0F0BD30B4842464005E
S31510003C500459284D254084246400055184246400A9
S31510003C600459254D25401C022C430C43D2B215068F
S31510003C70254384246400055130BC704730B4862433
S31510003C80640004591B4D2540862464000551862482
S31510003C9064000459194D25401C022C430C43D2B222
S31510003CA015062543802464052C4386256D00445152
S31510003CB030BC704710B504000848844203D1082070
S31510003CC0FFF733FC06E00848844203D18020C00287
S31510003CD0FFF72BFC10BD000000020048080000484A
S31510003CE0004000480042004808400048FF0300001A
S31510003CF0EF8000FCFFFFFFF8C0C0FFF8C0C0FFEF69
S31510003D00F0B540B2002821D5374C40B20207120F49
S31510003D10083A950804225543334A40B203071B0F4D
S31510003D20083B9B0804267343D258FF238607B60F19
S31510003D3008277E43B3409A438B01DBB28607B60F42
S31510003D4008277E43B340134363511AE0274A40B213
S31510003D50830804246343D258FF238407A40F08253D
S31510003D606C43A3409A438B01DBB28407A40F08254A
S31510003D706C43A34013431D4A40B2840804256C4388
S31510003D801351F0BD10B50400601E8021490488420D
S31510003D9001D301200EE0601E1549086003210020A2
S31510003DA0C043FFF7ADFF00201249086007201249F3
S31510003DB00860002010BD80B510480068FA218900FF
S31510003DC0FFF77AFBFFF7DEFF002000F001F801BDD8
S31510003DD00B49086070470A48006870470848006831
S31510003DE0401C0749086070471CED00E000E400E045
S31510003DF014E000E018E000E010E000E0D40100203C
S31510003E00CC01002080B523480068000AC0B22249C0
S31510003E1008602148006800282FD01E480068C0B2EC
S31510003E201E4908601D4800681D4909680902C0221C
S31510003E3092000A400243194802601948006880053A
S31510003E400CD41848144909688902144A126889184A
S31510003E50FFF732FB0001144908601AE0FFF782FBF6
S31510003E6080010D49096889020C4A12688918FFF702
S31510003E7023FB00010C4908600BE009480068800527
S31510003E8003D40A480849086003E0FFF76BFB0649AC
S31510003E90086001BD00030140C4010020C8010020D4
S31510003EA01C03014000001BB7D4010020006CDC028B
S31510003EB013008B404360704780B58022002116485E
S31510003EC000F030F8012200211348FFF7F1FF01BD81
S31510003ED010B5FFF780FF040010480068201AFA2179
S31510003EE04900884217D30E480078002809D10120CE
S31510003EF00B4908708022520200210748FFF7D8FFAD
S31510003F0007E0002006490870012200210248FFF749
S31510003F10CFFF0248046010BD00040440C001002019
S31510003F20D2010020F0B4C9B28B0804246343C3182D
S31510003F30C9B28C0804256C4304192469FC258E0724
S31510003F40B60F08277E43B540AC431C61C9B28B0837
S31510003F5004246343C418C9B28B0804256B43C318E1
S31510003F601D69D2B28E07B60F08235E431300B34005
S31510003F702B432361F0BC704780B5C0200849086008
S31510003F800848006808490140064801600748084982
S31510003F900860C32002490860FFF734FF01BD00BF67
S31510003FA0240001401C030140FFFDFFFF0001F13F0B
S31510003FB00003014070B40121002213E00468001DC3
S31510003FC00C4202D04D466D1E64192260241D1B1F23
S31510003FD0042BFAD225009E0701D52280AD1C0B407A
S31510003FE000D02A700368001D002BE7D170BC704703
S31510003FF010B5074979441831064C7C44163404E050
S31510004000081D0A68891888470100A142F8D110BD19
S3151000401008000000240000009DFFFFFF8000000044
S315100040205401002000000000F3F9FFFFFC0000001F
S315100040302E0100000C00002080B500F007F8FFF7F5
S3151000404007FBFFF745FFFFF709FBFAE780B5FFF718
S3151000405033FFFFF7B0FE01BD00F00BF8002801D0CA
S31510004060FFF7C6FF002000BF00BFFFF7E5FF00F017
S3151000407002F80120704780B500F002F801BDFEE796
S315100040800746384600F002F8FBE7FEE780B500BFAA
S3151000409000BF024A11001820ABBEFBE72600020043
S315100040A002488546024880470248004700400020E3
S315100040B0CD400010D9400010034800680121884304
S315100040C001490860704700BF6800014080B5FFF7DE
S315100040D0F3FFFFF751FF01BD00BF00BF00BF00BFD8
S315100040E0FFF7BAFFFEE7FEE7FEE7FEE7FEE7FEE7AD
S315100040F0FEE7FEE7FEE7FEE7FEE7FEE7FEE7FEE782
S31510004100FEE7FEE7FEE7FEE7FEE7FEE7FEE7FEE771
S31510004110FEE7FEE7FEE7FEE7FEE7FEE7FEE7FEE761
S31510004120FEE7FEE7FEE7FEE720022C4800470412F2
S315100041302B04122A041229041228041227045226C8
S3151000414004122404522308F1730410038B40001048
S315100041507F0412E50412E7041003DD3D0010E908A0
S3151000416012EB0412ED0412EF0412F10412F304120E
S31510004170F50412F70412F90412FB0412FD0412FFDF
S31510004180041003014100100304120504120704125F
S315100041900904120B04120D04120F04121104121347
S315100041A004121504121704121904121B04121D040A
S314100041B0121F04122104122304122504122704CD
S705100040D9D1
